:03000000020357A1
:03004300020100B7
:1001000002013C000201580002011800020129000E
:10011000020120000201180032E591C2E4F59122AB
:10012000C0E0C2003119D0E032C0E0E5874401F5FB
:10013000870000003119D0E032C2DC32C0D0C0E00C
:10014000C082C08312016931197401907FABF0D075
:1001500083D082D0E0D0D032C0D0C0E0C082C08393
:090160001203AF3119740280E2B0
:10016900907FE8E0A2E79202545C7051E0A2E0823D
:10017900E1404A30E50274035403C4F540A3E05456
:100189000F45401201D52001343002182003209078
:100199007F027846754003E6F0158218D540F8E6E7
:1001A900907FB5F0754002907FB4E04540F022851C
:1001B9008240E583907FD4F0E540A380E675400353
:1001C90080E5E02582F58250020583229001FA310B
:1001D900CCE09001FA31CCC082C0837845E4F618AE
:1001E900F6187601907FEAE0F5F0A3E0C201C203B8
:1001F900226D404040404081406A74404040404048
:1002090040714040404040A540404040404040404F
:1002190040714240404040404040404040404040A2
:1002290040405663404040404040435D404040406C
:1002390040D201223000FA907FC5F0907FAAE054A5
:100249000160FBF00203A13000E7087618223000B4
:10025900E0F541223000DA08A641223000D50876BF
:100269000122760222E5F060061470C5D20022C28E
:100279000022D203149002C560B9149002D760B36A
:100289001470AE900309E5F0601EF54031CBE060D3
:10029900A0E5401480F2D203C394219002E960934F
:1002A900149002F2608D8089E0FFF5F07800F20881
:0C02B900A3E0DFFAD0E0D0E0E5F021A9DE
:1002C500120101010000004042420001000101024B
:1002D500000109021B000101008032090400000031
:1002E500030000000921000100012217000600FF9C
:1002F5000901A10119012902150026FF00750895BC
:10030500039102C0040309042C0355005300420065
:100315002000440065007300690067006E0020003E
:100325004200790020004500780061006D007000F2
:100335006C0065001C0353007400650070007000BC
:100345006500720020004D006F0074006F007200A0
:1003550000007581EB75927F78D6E254F3F21203B3
:1003650090E24406F2E4F5207893E4F2799CF4F304
:1003750078ACF208F2087403F2087401F278AA74F2
:10038500FFF275E80175A8C00080FD75406490FB1B
:1003950050A3E582458370F9D540F3227846907ED7
:1003A500C07F03E0F6A308DFFA22D5492475490A80
:1003B50078477948E647601916E6F4600117E5467F
:1003C500700274FF2549540FF5499003D793789926
:1003D500F222070209101830292223262D343C1455
:0203E5000D0603
:00000001FF
